:100000000C9465000C948D000C948D000C948D0064
:100010000C948D000C948D000C948D000C94BC1DE0
:100020000C948D000C948D000C948D000C948D001C
:100030000C948D000C948D000C948D000C948D000C
:100040000C94A81A0C948D000C94101C0C948D0028
:100050000C948D000C948D000C948D000C948D00EC
:100060000C948D000C948D000200000000240027E9
:10007000002A0000000000250028002B00000000DE
:1000800000230026002900040404040404040402DC
:100090000202020202030303030303010204081025
:1000A00020408001020408102001020408102000F2
:1000B0000000070002010000030406000000000029
:1000C0000000000002030C1DFB0211241FBECFEF35
:1000D000D8E0DEBFCDBF11E0A0E0B1E0E0E2F8E49F
:1000E00002C005900D92AC35B107D9F713E0ACE52D
:1000F000B1E001C01D92A632B107E1F710E0C8ECF3
:10010000D0E004C02297FE010E94C023C43CD10766
:10011000C9F70E94461D0C9403240C940000CF9351
:10012000DF93BC018230910510F462E070E0A09191
:100130002403B0912503ED01E0E0F0E040E050E061
:1001400021C0888199818617970769F48A819B81EC
:10015000309719F09383828304C090932503809392
:100160002403FE0134C06817790738F4411551059E
:1001700019F08417950708F4AC01FE018A819B8170
:100180009C01E9012097E9F641155105A9F1CA0141
:10019000861B970B049708F4BA01E0E0F0E02AC050
:1001A0008D919C91119784179507F9F46417750741
:1001B00081F412968D919C911397309719F0938347
:1001C000828304C09093250380932403FD0132961B
:1001D0004CC0CA01861B970BFD01E80FF91F619304
:1001E000719302978D939C9340C0FD01828193810E
:1001F0009C01D9011097A1F68091220390912303CD
:10020000892B41F48091090190910A019093230375
:100210008093220340910B0150910C01411551052F
:1002200041F44DB75EB78091070190910801481BDA
:10023000590B2091220330912303CA01821B930B97
:100240008617970780F0AB014E5F5F4F84179507C5
:1002500050F0420F531F5093230340932203F901A0
:100260006193719302C0E0E0F0E0CF01DF91CF91A4
:100270000895CF93DF93009709F450C0EC012297C3
:100280001B821A82A0912403B0912503109709F1D3
:1002900040E050E0AC17BD0708F1BB83AA83FE0124
:1002A00021913191E20FF31FAE17BF0779F48D91C1
:1002B0009C911197280F391F2E5F3F4F3983288358
:1002C00012968D919C9113979B838A8341155105BA
:1002D00071F4D0932503C093240320C012968D910E
:1002E0009C911397AD01009711F0DC01D3CFFA0177
:1002F000D383C28321913191E20FF31FCE17DF0721
:1003000069F488819981280F391F2E5F3F4FFA01C8
:10031000318320838A819B8193838283DF91CF9174
:100320000895A0E0B0E0E7E9F1E00C94CE236C0181
:10033000009729F4CB010E948F006C01C1C08EEFA1
:10034000882E8FEF982E8C0C9D1C8601060F171F90
:100350000815190508F4B2C0F401A081B181A617EF
:10036000B707B8F0A530B10508F4AAC0CD010497CD
:100370008617970708F4A4C01297A61BB70BF801BD
:10038000A193B193D4016D937C93CF010E94390165
:1003900097C07B01EA1AFB0AEEEFFFEFEE0EFF1E9D
:1003A00036016A0E7B1EC0912403D091250344249C
:1003B0005524AA24BB244AC0C615D705E1F54881B7
:1003C00059814E155F05B8F1CA0104978E159F0536
:1003D000B0F41296A40FB51FF401B183A0832A8153
:1003E0003B814114510431F0D20113963C932E937A
:1003F000129766C0309325032093240361C08A813D
:100400009B81F80193838283425050404E195F09CB
:10041000518340834114510431F0D20113961C934F
:100420000E93129704C01093250300932403F40144
:100430007183608345C088819981A816B90608F444
:100440005C012E018A819B819C01E901209709F0C2
:10045000B3CF809122039091230386159705E9F489
:10046000A616B706D0F420910B0130910C0121158E
:10047000310541F42DB73EB78091070190910801F5
:10048000281B390B02171307C8F41093230300939A
:100490002203D4016D937C9313C0CB010E948F0083
:1004A000EC01009759F0F40140815181B6010E949E
:1004B0006602C6010E9439016E0102C0CC24DD240F
:1004C000C601CDB7DEB7E0E10C94EA23FB01DC0105
:1004D00002C001900D9241505040D8F70895FB01A1
:1004E000DC010D900020E9F7119701900D9200209A
:1004F000E1F70895FB01DC0101900D920020E1F786
:100500000895FA01CF93FF93EF932230CCF0253278
:10051000BCF4C22F2C2F332744275527FF93EF938A
:100520000E948123EF91FF91605D6A330CF0695D59
:100530006193B901CA01605070408040904051F70A
:1005400010828F919F91CF910C94A602DC01FC0147
:10055000672F71917723E1F7329704C07C916D93F7
:1005600070836291AE17BF07C8F308950F931F936E
:100570008C01FC01808191810E943901F801138274
:100580001282158214821F910F9108958130910576
:10059000E1F46F5F7F4F71F58CE691E060E071E010
:1005A0000E94392182E791E060E071E00E943921E8
:1005B00088E791E060E071E00E9439218EE791E0E8
:1005C00060E071E00E9439210895892B99F46F5FF2
:1005D0007F4F81F48EE791E00E94B60288E791E0B8
:1005E0000E94B60282E791E00E94B6028CE691E09A
:1005F0000E94B602089580E090E06FEF7FEF0E94C6
:10060000C602089581E090E06FEF7FEF0E94C6027E
:1006100008950F931F9309EF12E0C8016DE40E9443
:10062000F91CC8016DE40E94F91CC8016DE40E9428
:10063000F91CC80162E00E94F91CC80160915E01CA
:100640000E94F91C1F910F910895CF92DF92EF92B3
:10065000FF920F931F93DF93CF93CDB7DEB7CC56A6
:10066000D0400FB6F894DEBF0FBECDBF8BE068EE72
:1006700073E024E630E040E050E00E94181E8E0156
:100680000F5F1F4F8CE6F80111928A95E9F7809170
:100690005F01898390912C0280912D028A839B8334
:1006A00090912E0280912F028C839D839091340231
:1006B000809135028E839F83909132028091330224
:1006C0008887998790913002809131028A879B8731
:1006D00090914202809143028C879D8780916201B4
:1006E0008E8790913802809139028F87988B809104
:1006F0006001898B90914002809141028A8B9B8B93
:10070000809161018C8B80910D018D8B8BE692E045
:1007100065E170E00E944E188E8B8BE692E066E1F8
:1007200070E00E944E188F8B8BE692E067E170E0DC
:100730000E944E18888F8BE692E068E170E00E947C
:100740004E18898F8BE692E069E170E00E944E18A6
:100750008A8F8BE692E06AE170E00E944E188B8FE0
:100760008BE692E06BE170E00E944E188C8F8BE676
:1007700092E06CE170E00E944E188D8F8BE692E063
:100780006DE170E00E944E188E8F8BE692E06EE174
:1007900070E00E944E188F8F8BE692E06FE170E060
:1007A0000E944E1888A38BE692E060E270E00E94FF
:1007B0004E1889A38BE692E061E270E00E944E1829
:1007C0008AA38BE692E062E270E00E944E188BA34F
:1007D0008BE692E063E270E00E944E188CA38BE6F9
:1007E00092E064E270E00E944E188DA38BE692E0E6
:1007F00065E270E00E944E188EA38BE692E066E2FE
:1008000070E00E944E188FA38BE692E067E270E0E2
:100810000E944E1888A78BE692E068E270E00E9482
:100820004E1889A78BE692E069E270E00E944E18AC
:100830008AA78BE692E06AE270E00E944E188BA7CE
:100840008BE692E06BE270E00E944E188CA78BE67C
:1008500092E06CE270E00E944E188DA78BE692E069
:100860006DE270E00E944E188EA780910E018FA756
:100870008BE692E06FE270E00E944E1888AB8BE648
:1008800092E060E370E00E944E1889AB8BE692E044
:1008900061E370E00E944E188AAB8BE692E062E35F
:1008A00070E00E944E188BAB8BE692E063E370E041
:1008B0000E944E188CAB8BE692E064E370E00E94DD
:1008C0004E188DAB8BE692E065E370E00E944E1807
:1008D0008EAB8BE692E066E370E00E944E188FAB21
:1008E0008BE692E067E370E00E944E1888AF8BE6DB
:1008F00092E068E370E00E944E1889AF8091630136
:100900008AAF90913602809137028BAF9CAF809175
:1009100064018DAF90913A0280913B028EAF9FAF00
:1009200090913C0280913D02FE01E05CFF4F80838C
:10093000FE01EF5BFF4F9083909148028091490246
:10094000FE01EE5BFF4F8083FE01ED5BFF4F908366
:100950009091440280914502FE01EC5BFF4F808341
:10096000FE01EB5BFF4F908380916501FE01EA5B26
:10097000FF4F80839091460280914702FE01E95B20
:10098000FF4F8083FE01E85BFF4F90838091100151
:10099000FE01E75BFF4F80838BE692E069E470E045
:1009A0000E944E18FE01E65BFF4F80838BE692E0CB
:1009B0006AE470E00E944E18FE01E55BFF4F808301
:1009C0008BE692E06BE470E00E944E18FE01E45B5F
:1009D000FF4F80838BE692E06CE470E00E944E183B
:1009E000FE01E35BFF4F80838BE692E06DE470E0F5
:1009F0000E944E18FE01E25BFF4F80838BE692E07F
:100A00006EE470E00E944E18FE01E15BFF4F8083B0
:100A10008BE692E06FE470E00E944E18FE01E05B0E
:100A2000FF4F80838BE692E060E570E00E944E18F5
:100A3000FE01EF5AFF4F80838BE692E061E570E0A4
:100A40000E944E18FE01EE5AFF4F80838BE692E023
:100A500062E570E00E944E18FE01ED5AFF4F808360
:100A600080910F01FE01EC5AFF4F80838BE692E0EC
:100A700064E570E00E944E18FE01EB5AFF4F808340
:100A80008BE692E065E570E00E944E18FE01EA5A9E
:100A9000FF4F80838BE692E066E570E00E944E187F
:100AA000FE01E95AFF4F80838BE692E067E570E034
:100AB0000E944E18FE01E85AFF4F80838BE692E0B9
:100AC00068E570E00E944E18FE01E75AFF4F8083F0
:100AD0008BE692E069E570E00E944E18FE01E65A4E
:100AE000FF4F80838BE692E06AE570E00E944E182B
:100AF000FE01E55AFF4F80838BE692E06BE570E0E4
:100B00000E944E18FE01E45AFF4F80838BE692E06C
:100B10006CE570E00E944E18FE01E35AFF4F80839F
:100B20008BE692E06DE570E00E944E18FE01E25AFD
:100B3000FF4F808380916601FE01E15AFF4F808361
:100B400080916701FE01E05AFF4F80838091680128
:100B5000FE01EF59FF4F808380916901FE01EE593C
:100B6000FF4F808380916A01FE01ED59FF4F808322
:100B70009091120180911301FE01EC59FF4F808387
:100B8000FE01EB59FF4F908380915E02FE01EA590E
:100B9000FF4F808380915F02FE01E959FF4F808300
:100BA0009091630280916402FE01E859FF4F8083B7
:100BB000FE01E759FF4F908380916002FE01E659E4
:100BC000FF4F808380916102FE01E559FF4F8083D2
:100BD00080916202FE01E459FF4F808389EF92E029
:100BE0006DE30E94F91C89EF92E06DE30E94F91C0D
:100BF00089EF92E06DE30E94F91C78017DE6C72E33
:100C0000D12CCC0EDD1E89EF92E0F80161918F01AD
:100C10000E94F91C0C151D05B1F760E070E0562F1D
:100C2000472FF70181917F0190E0842795279C0150
:100C300064E0369527956A95E1F72F703070282784
:100C40003927C901982F88279295907F822793276B
:100C5000BC01707045E0660F771F4A95E1F7682781
:100C60007927E017F107D9F660933E0270933F02AF
:100C700089EF92E0672F0E94F91C89EF92E0609162
:100C80003E020E94F91CC459DF4F0FB6F894DEBF34
:100C90000FBECDBFCF91DF911F910F91FF90EF90CD
:100CA000DF90CF9008958F929F92BF92CF92DF9264
:100CB000EF92FF920F931F93DF93CF93CDB7DEB7E1
:100CC0002C970FB6F894DEBF0FBECDBF4C01162F88
:100CD000042F7E010894E11CF11CC70160E071E063
:100CE0000E943921B12EC12EDD24C00ED11C8E01EF
:100CF000095F1F4F10C08BE692E00E944E18682FCC
:100D0000C8010E94C620C701B8010E944A20C8013C
:100D10000E94B602B3946B2D70E06C157D055CF3F8
:100D2000C401B7010E946121C7010E94B602C4013B
:100D30002C960FB6F894DEBF0FBECDBFCF91DF91DA
:100D40001F910F91FF90EF90DF90CF90BF909F90F9
:100D50008F900895CF92DF92EF92FF920F931F939F
:100D6000DF93CF93CDB7DEB768970FB6F894DEBFA9
:100D70000FBECDBFF82E8BE692E060E070E00E94DF
:100D80004E18882311F481E010C08BE692E060E0F9
:100D900070E00E944E188D3310F08CE306C08BE695
:100DA00092E060E070E00E944E1880935F018BE655
:100DB00092E061E070E00E944E18182F8BE692E0FE
:100DC00062E070E00E944E18682F812F0E942E2052
:100DD0008436910518F484E690E028C08BE692E012
:100DE00061E070E00E944E18182F8BE692E062E0FE
:100DF00070E00E944E18682F812F0E942E20895B80
:100E00009B4018F088EB9BE011C08BE692E061E01C
:100E100070E00E944E18182F8BE692E062E070E0BE
:100E20000E944E18682F812F0E942E2090932D0231
:100E300080932C028BE692E063E070E00E944E18F3
:100E4000182F8BE692E064E070E00E944E18682F45
:100E5000812F0E942E208BE692E063E070E00E94DA
:100E60004E18182F8BE692E064E070E00E944E1856
:100E7000682F812F0E942E20895E934018F088EE03
:100E800093E011C08BE692E063E070E00E944E18A0
:100E9000182F8BE692E064E070E00E944E18682FF5
:100EA000812F0E942E2090932F0280932E028BE69A
:100EB00092E065E070E00E944E18182F8BE692E0F9
:100EC00066E070E00E944E18682F812F0E942E204D
:100ED0008BE692E065E070E00E944E18182F8BE6DA
:100EE00092E066E070E00E944E18682F812F0E9409
:100EF0002E20895E934018F088EE93E011C08BE6B7
:100F000092E065E070E00E944E18182F8BE692E0A8
:100F100066E070E00E944E18682F812F0E942E20FC
:100F200090933502809334028BE692E067E070E0A4
:100F30000E944E18182F8BE692E068E070E00E9445
:100F40004E18682F812F0E942E204E9718F48EE1A4
:100F500090E028C08BE692E067E070E00E944E18B7
:100F6000182F8BE692E068E070E00E944E18682F20
:100F7000812F0E942E208D52914018F08CE291E03A
:100F800011C08BE692E067E070E00E944E18182FC7
:100F90008BE692E068E070E00E944E18682F812F87
:100FA0000E942E2090933302809332028BE692E0CF
:100FB00069E070E00E944E18182F8BE692E06AE01C
:100FC00070E00E944E18682F812F0E942E208C52B4
:100FD000914018F48CE291E028C08BE692E069E041
:100FE00070E00E944E18182F8BE692E06AE070E0E5
:100FF0000E944E18682F812F0E942E208D5D9540F3
:1010000018F08CED95E011C08BE692E069E070E09D
:101010000E944E18182F8BE692E06AE070E00E9462
:101020004E18682F812F0E942E20909331028093BA
:1010300030028BE692E06BE070E00E944E18182FB1
:101040008BE692E06CE070E00E944E18682F812FD2
:101050000E942E208C52914018F48CE291E028C01E
:101060008BE692E06BE070E00E944E18182F8BE642
:1010700092E06CE070E00E944E18682F812F0E9471
:101080002E20815D974018F080ED97E011C08BE62F
:1010900092E06BE070E00E944E18182F8BE692E011
:1010A0006CE070E00E944E18682F812F0E942E2065
:1010B00090934302809342028BE692E06DE070E0F1
:1010C0000E944E188BE692E06DE070E00E944E1890
:1010D0008F3110F08EE106C08BE692E06DE070E09B
:1010E0000E944E18809362018BE692E06EE070E001
:1010F0000E944E18182F8BE692E06FE070E00E947D
:101100004E18682F812F0E942E208BE692E06EE011
:1011100070E00E944E18182F8BE692E06FE070E0AE
:101120000E944E18682F812F0E942E20895E9340C6
:1011300018F088EE93E011C08BE692E06EE070E06C
:101140000E944E18182F8BE692E06FE070E00E942C
:101150004E18682F812F0E942E2090933902809381
:1011600038028BE692E060E170E00E944E1888231E
:1011700011F481E010C08BE692E060E170E00E9423
:101180004E188F3110F08EE106C08BE692E060E1E0
:1011900070E00E944E18809360018BE692E061E15E
:1011A00070E00E944E18182F8BE692E062E170E02A
:1011B0000E944E18682F812F0E942E208C52914041
:1011C00018F48CE291E028C08BE692E061E170E0D7
:1011D0000E944E18182F8BE692E062E170E00E94A8
:1011E0004E18682F812F0E942E20815D974018F0A5
:1011F00080ED97E011C08BE692E061E170E00E9423
:101200004E18182F8BE692E062E170E00E944E18B3
:10121000682F812F0E942E209093410280934002DC
:101220008BE692E063E170E00E944E18833010F488
:1012300083E010C08BE692E063E170E00E944E18FC
:10124000853B10F084EB06C08BE692E063E170E032
:101250000E944E18809361018BE692E064E170E099
:101260000E944E188BE692E064E170E00E944E18F6
:101270008A3110F049E107C08BE692E064E170E04A
:101280000E944E18482F40930D018E010F5F1F4F93
:10129000C80165E10E9453068CE691E0B8010E9406
:1012A0009620C8010E94B6028BE692E06EE270E0E2
:1012B0000E944E188BE692E06EE270E00E944E189B
:1012C0008B3010F04AE007C08BE692E06EE270E0EF
:1012D0000E944E18482F40930E018E01095F1F4F48
:1012E000C8016FE20E9453068EE791E0B8010E94A8
:1012F0009620C8010E94B6028BE692E069E370E096
:101300000E944E18882311F481E010C08BE692E011
:1013100069E370E00E944E18853110F084E106C048
:101320008BE692E069E370E00E944E1880936301BF
:101330008BE692E06AE370E00E944E18182F8BE66D
:1013400092E06BE370E00E944E18682F812F0E949C
:101350002E208C52914018F48CE291E028C08BE64C
:1013600092E06AE370E00E944E18182F8BE692E03C
:101370006BE370E00E944E18682F812F0E942E2090
:101380008D5D954018F08CED95E011C08BE692E0F4
:101390006AE370E00E944E18182F8BE692E06BE330
:1013A00070E00E944E18682F812F0E942E2090938B
:1013B0003702809336028BE692E06CE370E00E9485
:1013C0004E188E3010F48EE010C08BE692E06CE385
:1013D00070E00E944E188E3210F08DE206C08BE64F
:1013E00092E06CE370E00E944E18809364018BE6FB
:1013F00092E06DE370E00E944E18182F8BE692E0A9
:101400006EE370E00E944E18682F812F0E942E20FC
:101410008BE692E06DE370E00E944E18182F8BE689
:1014200092E06EE370E00E944E18682F812F0E94B8
:101430002E20895E934018F088EE93E011C08BE671
:1014400092E06DE370E00E944E18182F8BE692E058
:101450006EE370E00E944E18682F812F0E942E20AC
:1014600090933B0280933A028BE692E06FE370E048
:101470000E944E18182F8BE692E060E470E00E9404
:101480004E18682F812F0E942E208BE692E06FE38A
:1014900070E00E944E18182F8BE692E060E470E036
:1014A0000E944E18682F812F0E942E20895E934043
:1014B00018F088EE93E011C08BE692E06FE370E0E5
:1014C0000E944E18182F8BE692E060E470E00E94B4
:1014D0004E18682F812F0E942E2090933D028093FA
:1014E0003C028BE692E061E470E00E944E18182FF7
:1014F0008BE692E062E470E00E944E18682F812F24
:101500000E942E208BE692E061E470E00E944E186B
:10151000182F8BE692E062E470E00E944E18682F6C
:10152000812F0E942E208BE692E061E470E00E9401
:101530004E18182F8BE692E062E470E00E944E187D
:10154000682F812F0E942E20909349028093480299
:101550008BE692E063E470E00E944E18182F8BE651
:1015600092E064E470E00E944E18682F812F0E9480
:101570002E208858934118F488E893E128C08BE620
:1015800092E063E470E00E944E18182F8BE692E020
:1015900064E470E00E944E18682F812F0E942E2074
:1015A00081589E4318F080E89EE311C08BE692E0DC
:1015B00063E470E00E944E18182F8BE692E064E41A
:1015C00070E00E944E18682F812F0E942E20909369
:1015D0004502809344028BE692E066E470E00E944C
:1015E0004E18182F8BE692E067E470E00E944E18C8
:1015F000682F812F0E942E208BE692E066E470E037
:101600000E944E18182F8BE692E067E470E00E946B
:101610004E18682F812F0E942E208BE692E066E400
:1016200070E00E944E18182F8BE692E067E470E09D
:101630000E944E18682F812F0E942E2090934702FF
:10164000809346028BE692E068E470E00E944E18B8
:101650008BE692E068E470E00E944E188B3010F048
:101660004AE007C08BE692E068E470E00E944E1802
:10167000482F409310018E01035F1F4FC80169E49A
:101680000E94530688E791E0B8010E949620C801A5
:101690000E94B6028BE692E063E570E00E944E186D
:1016A0008BE692E063E570E00E944E188B3010F0FC
:1016B0004AE007C08BE692E063E570E00E944E18B6
:1016C000482F40930F018E010D5E1F4FC80164E546
:1016D0000E94530682E791E0B8010E949620C8015B
:1016E0000E94B6028BE692E06EE570E00E944E1812
:1016F0008BE692E06EE570E00E944E188BE692E079
:101700006EE570E00E944E18809366018BE692E0D1
:101710006FE570E00E944E188BE692E06FE570E096
:101720000E944E188BE692E06FE570E00E944E1822
:10173000809367018BE692E060E670E00E944E18AD
:101740008BE692E060E670E00E944E188BE692E035
:1017500060E670E00E944E18809368018BE692E08C
:1017600061E670E00E944E188BE692E061E670E060
:101770000E944E1887FF02C08FE706C08BE692E0FA
:1017800061E670E00E944E18809369018BE692E05A
:1017900062E670E00E944E188BE692E062E670E02E
:1017A0000E944E188BE692E062E670E00E944E18AE
:1017B00080936A018BE692E063E670E00E944E1827
:1017C0008BE692E063E670E00E944E18803210F0E3
:1017D0008FE106C08BE692E063E670E00E944E184F
:1017E00080935E028BE692E064E670E00E944E1801
:1017F000882311F481E010C08BE692E064E670E08B
:101800000E944E188D3010F08CE006C08BE692E0FE
:1018100064E670E00E944E1880935F028BE692E0CF
:1018200065E670E00E944E18182F8BE692E066E69F
:1018300070E00E944E18682F812F0E942E208BE6A8
:1018400092E065E670E00E944E18182F8BE692E059
:1018500066E670E00E944E18682F812F0E942E20AD
:10186000895B9B4018F088EB9BE011C08BE692E00F
:1018700065E670E00E944E18182F8BE692E066E64F
:1018800070E00E944E18682F812F0E942E209093A6
:101890006402809363028BE692E067E670E00E9448
:1018A0004E188BE692E067E670E00E944E18893190
:1018B00010F088E106C08BE692E067E670E00E94D7
:1018C0004E18809360028BE692E068E670E00E941A
:1018D0004E188BE692E068E670E00E944E188C335A
:1018E00010F08BE306C08BE692E068E670E00E94A1
:1018F0004E18809361028BE692E069E670E00E94E8
:101900004E188BE692E069E670E00E944E188C3328
:1019100010F08BE306C08BE692E069E670E00E946F
:101920004E1880936202FF2011F188E390E00E943C
:101930009419F82EE92EC0903602D09037026091AB
:10194000640170E080E090E00E9439228B019C01EC
:101950008F2D9E2D6BE070E0A6010E948E1AF092F2
:101960005C02E0925D028F2D9E2D0E94661A8BE034
:1019700060ED77E024E630E040E050E00E94181E81
:1019800068960FB6F894DEBF0FBECDBFCF91DF9142
:101990001F910F91FF90EF90DF90CF9008951F93CC
:1019A000182F86E0612F0E94B81B80914802909109
:1019B000490297FF03C0112319F004C0112311F04D
:1019C000419A01C041981F910895682F85E00E94B7
:1019D000B81B08950F931F93CF93DF932091660256
:1019E000E22FF0E0E455FE4F80832F5F20936602E4
:1019F0008091AC01A82FB0E0BD016F5F7F4F30E058
:101A0000621773070CF0ABC01092660210925D0172
:101A100010925C01ECEAF1E0C0E0D0E08D010E0F25
:101A20001F1F20C05C2F4D2F819190E084279527A8
:101A30009C0154E0369527955A95E1F72F70307048
:101A400028273927C901982F88279295907F8227C8
:101A50009327EC01D07025E0CC0FDD1F2A95E1F72C
:101A6000C827D927E017F107E9F6C0933E02D093C3
:101A70003F02A455BE4F64557E4F8C91FB0160819F
:101A80000E942E20C817D90709F069C08091AD01C6
:101A900080936502833109F448C0843128F4813190
:101AA00049F08231C9F53AC0843109F44AC0853120
:101AB00099F54AC010E00BC0E12FF0E08BE692E010
:101AC000BF01E455FE4F42810E9455181F5F80916F
:101AD000AC01181788F380915C0290915D020E941E
:101AE000971990E0882309F491E0892F0E94AA06B3
:101AF00089EF92E061EF0E94F91C89EF92E061EFBB
:101B00000E94F91C89EF92E061EF0E94F91C89EFB5
:101B100092E06FEF0E94F91C80E019C081E00E9402
:101B2000E50C80911101877F06C080E00E94E50CE2
:101B300080911101886080931101809580935E01EE
:101B4000EBCF0E942503E8CF0E940903E5CFE82FE1
:101B5000F0E0E455FE4F10828F5F8038C1F7DF91CF
:101B6000CF911F910F91089520915C0130915D01FB
:101B70002130310591F0223031051CF4232B41F046
:101B800008952230310571F023303105D9F418C0A1
:101B90008A3289F481E090E009C08A3261F482E0FF
:101BA00090E004C08A3239F483E090E090935D01C4
:101BB00080935C01089510925D0110925C0108957C
:101BC0000E94EA0C0895EF92FF920F931F930E94D8
:101BD000F01A60938401709385018093860190933D
:101BE000870189EF92E00E949E1C892BE1F0809191
:101BF000840190918501A0918601B0918701809325
:101C0000880190938901A0938A01B0938B0189EF99
:101C100092E00E94C91C0E94B40D61E070E080E077
:101C200090E00E94FE1A209184013091850140913C
:101C30008601509187018091880190918901A0913E
:101C40008A01B0918B0179018A01E81AF90A0A0B1D
:101C50001B0BD801C701855F9140A040B04060F0E8
:101C600010925D0110925C012093880130938901EC
:101C700040938A0150938B011F910F91FF90EF9039
:101C80000895EF92FF920F931F93DF93CF93CDB7F9
:101C9000DEB72C970FB6F894DEBF0FBECDBF809194
:101CA0004D02882361F18BE068E572E026E430E0C4
:101CB00040E050E00E94181E66E470E080E090E092
:101CC0000E94FE1A8BE060E273E026E430E040E020
:101CD00050E00E94181E66E470E080E090E00E94F0
:101CE000FE1A8BE06CE474E028EC30E040E050E059
:101CF0000E94181E10924D0210924E0264C08091F4
:101D00004E028823F1F0E0905C02F0905D028E01BB
:101D10000F5F1F4FC80161E071E00E943921C701C8
:101D2000B8010E944F1AC8010E94B60280915C025D
:101D300090915D020E94291A10924E0210924D025B
:101D400042C080914F02882369F1609142027091F4
:101D500043028BE02CE330E040E050E00E94181E8C
:101D600066E470E080E090E00E94FE1A209142025A
:101D700030914302C90164E670E00E946D2389E15D
:101D800090E0AC01649FC001659F900D749F900D21
:101D90001124281B390B8BE0B9012CE330E040E023
:101DA00050E00FC08091480282FF0DC06091300268
:101DB00070913102209132023091330240E050E0C4
:101DC0008BE00E94181E809150028823F9F0E09069
:101DD0005C02F0905D028E01095F1F4F609112015D
:101DE00070911301C8014AE050E00E94FB20C70136
:101DF000B8010E944F1AC8010E94B60280915C028D
:101E000090915D020E94291A109250022C960FB6F2
:101E1000F894DEBF0FBECDBFCF91DF911F910F9120
:101E2000FF90EF9008950F931F93182F092FCB0168
:101E3000BA010E944A20BC01812F902F0E94E0200D
:101E4000812F902F1F910F9108952F923F924F92C3
:101E50005F926F927F928F929F92AF92BF92CF923A
:101E6000DF92EF92FF920F931F93DF93CF93CDB743
:101E7000DEB7C257D0400FB6F894DEBF0FBECDBF5D
:101E80000E94F01A9B01AC01609390017093910144
:101E90008093920190939301329904C080914802FB
:101EA00080FD06C0339913C08091480281FF0FC0A6
:101EB00080916702882359F42093A4013093A501EF
:101EC0004093A6015093A70181E08093670280911F
:101ED0006702882311F40C94C817329B02C00C943B
:101EE000C8178091480280FD02C00C94C817209149
:101EF0009001309191014091920150919301809114
:101F0000A4019091A501A091A601B091A701281B61
:101F1000390B4A0B5B0B80913A0290913B02A0E097
:101F2000B0E082179307A407B50710F00C94C81708
:101F300091E090934A02809152028823D9F48091D3
:101F400011018F7780931101809580935E019093AA
:101F5000520210C010924A0280915202882351F01E
:101F600080911101806880931101809580935E01BA
:101F70001092520280916702882311F40C94CE17BC
:101F8000339B02C00C94CE178091480281FD02C0A1
:101F90000C94CE17209190013091910140919201C3
:101FA000509193018091A4019091A501A091A60167
:101FB000B091A701281B390B4A0B5B0B80913C02A7
:101FC00090913D02A0E0B0E082179307A407B50707
:101FD00008F0E4C791E090934A028091510288236F
:101FE000D9F4809111018F7B8093110180958093AA
:101FF0005E019093510210C010924A0280915102EA
:10200000882351F0809111018064809311018095A3
:1020100080935E0110925102809167028823C1F182
:10202000329936C0209190013091910140919201F6
:10203000509193018091A4019091A501A091A601D6
:10204000B091A701281B390B4A0B5B0B80912E0224
:1020500090912F0260913A0270913B02860F971F78
:10206000A0E0B0E082179307A407B50788F491E0D9
:1020700090934C0280915302882351F48091110176
:102080008F7D80931101809580935E019093530220
:10209000809167028823C1F1339936C02091900165
:1020A0003091910140919201509193018091A4014E
:1020B0009091A501A091A601B091A701281B390B11
:1020C0004A0B5B0B80912E0290912F0260913C0293
:1020D00070913D02860F971FA0E0B0E08217930732
:1020E000A407B50788F491E090934C0280915302C5
:1020F000882351F4809111018F7D80931101809587
:1021000080935E0190935302809167028823C1F10E
:10211000329936C020919001309191014091920105
:10212000509193018091A4019091A501A091A601E5
:10213000B091A701281B390B4A0B5B0B80912C0235
:1021400090912D0260913A0270913B02860F971F89
:10215000A0E0B0E082179307A407B50788F491E0E8
:1021600090934B0280915402882351F48091110185
:102170008D7F80931101809580935E01909354022E
:10218000809167028823C1F1339936C02091900174
:102190003091910140919201509193018091A4015D
:1021A0009091A501A091A601B091A701281B390B20
:1021B0004A0B5B0B80912C0290912D0260913C02A6
:1021C00070913D02860F971FA0E0B0E08217930741
:1021D000A407B50788F491E090934B0280915402D4
:1021E000882351F4809111018D7F80931101809596
:1021F00080935E0190935402329B04C0339B02C0D3
:102200001092670280914B02882309F4E2C3809107
:102210004A02882309F44DC080915602882399F41C
:1022200081E00E94CF0C809111018E7F809311017B
:10223000809580935E0190E080915602882309F496
:1022400091E090935602809155028823B9F48091D1
:102250005902882399F481E00E94E50C80911101D4
:10226000877F80931101809580935E0190E080913B
:102270005502882309F491E09093550281E0809300
:1022800069028091900190919101A0919201B09189
:1022900093018093940190939501A0939601B0933C
:1022A00097018093980190939901A0939A01B0931C
:1022B0009B0180914A02882309F097C080916902AE
:1022C000813009F092C020919001309191014091AC
:1022D0009201509193018091940190919501A09168
:1022E0009601B0919701281B390B4A0B5B0B80912B
:1022F000340290913502A0E0B0E082179307A40762
:10230000B50708F072C080915A028823C1F080910D
:102310005C0290915D026AE270E00E947319809104
:102320001101806180931101809580935E0190E09E
:1023300080915A02882309F491E090935A02809187
:102340006B018330E9F48091480287FF19C0E09067
:102350005C02F0905D028E010F5F1F4FC80161E0CB
:1023600071E00E943921C701B8010E944F1AC801CB
:102370000E94B60280915C0290915D020E94291A2F
:1023800080915C0290915D020E949719882331F43C
:1023900080914C02882311F00E94410E82E08093CC
:1023A00069028091900190919101A0919201B09168
:1023B000930180939C0190939D01A0939E01B09303
:1023C0009F0110924C021092590210926B01809161
:1023D0005302882351F08091110180628093110192
:1023E000809580935E011092530280914A02882367
:1023F00009F054C080916902823009F04FC0E0902A
:102400009001F090910100919201109193018091BF
:10241000940190919501A0919601B0919701E81ACD
:10242000F90A0A0B1B0B8091320290913302209122
:10243000340230913502820F931F2091620130E007
:1024400048EE53E0B901649F9001659F300D749F81
:10245000300D1124820F931FA0E0B0E08E159F0570
:10246000A007B107D8F480915502882399F080E045
:102470000E94E50C80911101886080931101809584
:1024800080935E0190E080915502882309F491E0E9
:10249000909355021092690210925802809048025F
:1024A00085FEF4C180916902813009F0EFC180910D
:1024B0006702882309F48AC0A0909001B09091012E
:1024C000C0909201D09093018091A4019091A501B8
:1024D000A091A601B091A70186017501E81AF90A39
:1024E0000A0B1B0B6091600170E080E090E020E639
:1024F0003AEE40E050E00E944E2320913A023091A3
:102500003B0240E050E0620F731F841F951F209133
:10251000610130E048EE53E0D901A49F9001A59FEE
:10252000300DB49F300D1124442737FD4095542FB2
:10253000621B730B840B950B6E157F05800791074B
:1025400008F044C08091A8019091A901A091AA012E
:10255000B091AB01A81AB90ACA0ADB0AB9EEAB16E8
:10256000B3E0BB06B0E0CB06B0E0DB0678F18091CB
:102570006B01882359F586FE29C080915A02882371
:1025800051F08091110180618093110180958093B9
:102590005E0110925A0260914002709141028BE0FC
:1025A0002EE130E040E050E00E94181E8091900142
:1025B00090919101A0919201B09193018093A80113
:1025C0009093A901A093AA01B093AB0180916702F7
:1025D000882309F454C0A0909001B0909101C0905C
:1025E0009201D09093018091A4019091A501A091B6
:1025F000A601B091A701A81AB90ACA0ADB0AE0909D
:102600003A02F0903B0200E010E068E17CEF8FEFCF
:102610009FEFE60EF71E081F191F6091600170E022
:1026200080E090E020E63AEE40E050E00E944E2349
:10263000E60EF71E081F191FEA14FB040C051D0502
:10264000F0F480916B018823D1F480915A028823A1
:1026500051F08091110180618093110180958093E8
:102660005E0110925A028BE068EE73E024E630E0DF
:1026700040E050E00E94181E81E080936B01809141
:102680006702882309F454C0A0909001B090910192
:10269000C0909201D09093018091A4019091A501E6
:1026A000A091A601B091A701A81AB90ACA0ADB0A2B
:1026B000E0903A02F0903B0200E010E080EE9CEFE8
:1026C000AFEFBFEFE80EF91E0A1F1B1F60916001FC
:1026D00070E080E090E020E63AEE40E050E00E94BA
:1026E0004E23E60EF71E081F191FEA14FB040C0503
:1026F0001D05F0F480916B018130D1F480915A0274
:10270000882351F08091110180618093110180959F
:1027100080935E0110925A028BE060E273E024E63F
:1027200030E040E050E00E94181E82E080936B0190
:1027300080916702882309F454C0A0909001B09062
:102740009101C0909201D09093018091A401909149
:10275000A501A091A601B091A701A81AB90ACA0AB9
:10276000DB0AE0903A02F0903B0200E010E068EAF9
:102770007DEF8FEF9FEFE60EF71E081F191F609188
:10278000600170E080E090E020E63AEE40E050E04A
:102790000E944E23E60EF71E081F191FEA14FB04C1
:1027A0000C051D05F0F480916B018230D1F480910D
:1027B0005A02882351F080911101806180931101A8
:1027C000809580935E0110925A028BE068E572E07A
:1027D00028EC30E040E050E00E94181E83E0809337
:1027E0006B0180916702882309F450C0E09090014A
:1027F000F090910100919201109193018091A401B8
:102800009091A501A091A601B091A701E81AF90A3B
:102810000A0B1B0B6091600170E080E090E020E605
:102820003AEE40E050E00E944E2320913A0230916F
:102830003B0240E050E0260F371F481F591F2E155E
:102840003F054007510710F580916B018330F1F48B
:10285000809159028823D1F40E94E50C80911101E6
:10286000886080931101809580935E0190E0809153
:102870005902882309F491E09093590290E08091E5
:102880005502882309F491E09093550280914A0201
:102890008823B1F5209190013091910140919201EE
:1028A000509193018091980190919901A0919A0182
:1028B000B0919B01281B390B4A0B5B0B80913802AE
:1028C00090913902A0E0B0E082179307A407B50702
:1028D000B8F480915602882399F080E00E94CF0CD2
:1028E00080911101816080931101809580935E0138
:1028F00090E080915602882309F491E0909356026B
:1029000080914A02882381F580916902813061F5C6
:102910008091900190919101A0919201B0919301C9
:102920002091940130919501409196015091970129
:10293000821B930BA40BB50B87399105A105B1053B
:1029400098F080916B01833079F48091480287FF81
:102950000BC081E00E94E50C80911101877F80937C
:102960001101809580935E01E0909001F0909101BB
:102970000091920110919301809198019091990199
:10298000A0919A01B0919B01E81AF90A0A0B1B0B5E
:1029900060915F0170E080E090E020E63AEE40E078
:1029A00050E00E944E236E157F058007910798F432
:1029B00010924B0280915402882369F0809111019A
:1029C000826080931101809580935E011092540281
:1029D00002C010924C0280916802882309F0B5C0B1
:1029E00080916902823009F0B0C02091900130914D
:1029F0009101409192015091930180919C0190919D
:102A00009D01A0919E01B0919F01281B390B4A0B9B
:102A10005B0B80913402909135026091320270918B
:102A20003302860F971F8C509E4FA0E0B0E08217B4
:102A30009307A407B50708F088C08091480283FF78
:102A400084C020905C0230905D0267E0462E512CDD
:102A50004C0E5D1EC2016CE671E00E94E0205DE05C
:102A6000652E712C6C0E7D1EC30163E071E00E9427
:102A7000392143E1842E912C8C0E9D1EC401B2019C
:102A8000A3010E94130F39E1A32EB12CAC0EBD1E81
:102A9000C501B40142E751E00E94130F2FE1C22E9D
:102AA000D12CCC0EDD1EC60163E071E00E943921FD
:102AB00095E2E92EF12CEC0EFD1EC701B501A60131
:102AC0000E94130F8E01055D1F4FC801B70148E733
:102AD00051E00E94130FC101B8010E944F1AC801B2
:102AE0000E94B602C7010E94B602C6010E94B60249
:102AF000C5010E94B602C4010E94B602C3010E9431
:102B0000B602C2010E94B60280915C0290915D0201
:102B10000E94291A8091900190919101A0919201B7
:102B2000B091930180939C0190939D01A0939E018D
:102B3000B0939F018093A0019093A101A093A20163
:102B4000B093A30181E080936802E0909001F0903F
:102B500091010091920110919301809198019091BF
:102B60009901A0919A01B0919B01E81AF90A0A0B08
:102B70001B0B6091630170E080E090E020E63AEE8C
:102B800040E050E00E944E236E157F0580079107BC
:102B900020F4109268021092690280910D0188233E
:102BA00009F44FC0E0909001F090910100919201E2
:102BB000109193018091A0019091A101A091A20197
:102BC000B091A301E81AF90A0A0B1B0B609163018B
:102BD00070E080E090E020E63AEE40E050E00E94B5
:102BE0004E23645F7140804090406E157F058007E2
:102BF000910738F580916802813019F5809148027B
:102C000083FF1FC080916B018823D9F48091550206
:102C10008823B9F480915802882399F481E00E94B6
:102C2000E50C80911101877F80931101809580933D
:102C30005E0190E080915802882309F491E090931E
:102C4000580280910D01882309F484C0E09090011E
:102C5000F090910100919201109193018091A00157
:102C60009091A101A091A201B091A301E81AF90AE3
:102C70000A0B1B0B6091630170E080E090E020E69E
:102C80003AEE40E050E00E944E236E157F0580072B
:102C9000910708F05FC080916802813009F05AC046
:102CA0008091480283FF56C080916B01882309F010
:102CB00051C080905C0290905D0281E3A82EB12CFF
:102CC000AC0EBD1EC5016CE671E00E94E02007E37A
:102CD000C02ED12CCC0EDD1EC60163E071E00E9437
:102CE00039211DE3E12EF12CEC0EFD1EC701B501CB
:102CF000A6010E94130F8E010D5B1F4FC801B70183
:102D000048E751E00E94130FC401B8010E944F1A16
:102D1000C8010E94B602C7010E94B602C6010E9405
:102D2000B602C5010E94B60280915C0290915D02DC
:102D30000E94291A8091900190919101A091920195
:102D4000B09193018093A0019093A101A093A2015F
:102D5000B093A30180915C0290915D020E9497194B
:102D6000882339F180915702882399F481E00E94E9
:102D7000E50C80911101877F8093110180958093EC
:102D80005E0190E080915702882309F491E09093CE
:102D900057028091900190919101A0919201B09180
:102DA00093018093940190939501A0939601B09321
:102DB000970180915C0290915D020E94971988238F
:102DC000E1F4809157028823C1F080916902882341
:102DD000A1F40E94E50C809111018860809311019B
:102DE000809580935E0190E080915702882309F4DA
:102DF00091E0909357021092580280915C0290915A
:102E00005D020E949719882309F180914A02882364
:102E1000E9F080915A028823C9F46091640180919D
:102E20005C0290915D0270E00E9473198091110123
:102E30008F7E80931101809580935E0190E0809158
:102E40005A02882309F491E090935A028091670214
:102E5000882309F4A6C08091900190919101A091DE
:102E60009201B09193012091A4013091A50140916C
:102E7000A6015091A701821B930BA40BB50B8151A6
:102E80009742A040B04008F48CC08091480283FF74
:102E900088C080915B02882309F083C0809168021A
:102EA000882309F07EC020905C0230905D02B9E476
:102EB0004B2E512C4C0E5D1EC2016CE671E00E943F
:102EC000E020AFE46A2E712C6C0E7D1EC30163E01E
:102ED00071E00E943921F5E58F2E912C8C0E9D1EFC
:102EE000C401B201A3010E94130FEBE5AE2EB12C79
:102EF000AC0EBD1EC501B40142E751E00E94130FA4
:102F000071E6C72ED12CCC0EDD1EC60163E071E048
:102F10000E94392167E6E62EF12CEC0EFD1EC7015A
:102F2000B501A6010E94130F8E0103591F4FC8015E
:102F3000B70148E751E00E94130FC101B8010E9498
:102F40004F1AC8010E94B602C7010E94B602C6010C
:102F50000E94B602C5010E94B602C4010E94B602D8
:102F6000C3010E94B602C2010E94B60280915C02B7
:102F700090915D020E94291A90E080915B02882363
:102F800009F491E090935B0281E08093680209C0AC
:102F9000339B02C00C94AA0F0C94BA0F32992CC820
:102FA0003BC8CE58DF4F0FB6F894DEBF0FBECDBF83
:102FB000CF91DF911F910F91FF90EF90DF90CF9015
:102FC000BF90AF909F908F907F906F905F904F9049
:102FD0003F902F9008950E94E30D0E94250F0E94BC
:102FE000F01A20918C0130918D0140918E01509109
:102FF0008F01621B730B840B950B655F71408040E2
:10300000904048F10E94F01A60938C0170938D01FA
:1030100080938E0190938F0160916A02662321F460
:10302000809111018B7F05C0613029F480911101DD
:1030300084608093110180911101809580935E01DD
:103040008AE00E94B81B90E080916A02882309F40C
:1030500091E090936A02089589EF92E040E051EE8A
:1030600060E070E00E94411C81E00E94AA0685E0B9
:1030700061E00E94921B80E00E94E50C8AE061E022
:103080000E94921B86E061E00E94921B86E060E055
:103090000E94B81B399A429A439A0895F999FECF33
:1030A00072BD61BDF89A80B50895F999FECF1FBA37
:1030B00072BD61BD40BD0FB6F894FA9AF99A0FBE81
:1030C0000895FF920F931F93CF93DF93EC018B0131
:1030D000A0E0B0E0FF2430E860E070E050E020E0E5
:1030E000832F90E084239523181619060CF421E011
:1030F000FF2029F42223F9F0FF24F3941CC022239B
:1031000019F08E819F8102C08C819D81FD01EE0F9F
:10311000FF1FEE0FFF1FE00FF11F91838083FD0162
:10312000EE0FFF1FEE0FFF1FE00FF11F8C819D813F
:1031300093838283119636956F5F7F4F6830710558
:1031400071F6CD01DF91CF911F910F91FF900895FE
:10315000CF93DF93EC01962F862F81568A3160F44E
:10316000BE01625F7F4FE92FFF27E7FDF095EC532B
:10317000FF4FCE01408149C0862F80538A3028F00E
:10318000EFE3F1E0A0E0B0E047C0772767FD70957E
:103190009B012053304080E02630310514F481E05B
:1031A00003C09B0125533040DE01E0E0F0E0482FF2
:1031B00050E080E090E0E217F30714F481E090E043
:1031C0008417950719F48C819D8102C08E819F819F
:1031D0001F969C938E931E978C819D8151969C93F4
:1031E0008E93509731961496E530F10511F710C083
:1031F0003296891781F4BE01625F7F4FAA0FBB1F11
:10320000A15CBE4FCE0111964C910E946118FC0149
:1032100020E030E008C011968081882349F7E1E082
:10322000F0E021E030E0EE0FFF1F3696DF01AA0F3D
:10323000BB1FAC0FBD1F8E819F818D939C933196D8
:10324000EE0FFF1FEC0FFD1F11821082F901379660
:10325000EE0FFF1FEC0FFD1F81919191892BE1F77C
:10326000C901DF91CF91089508950895EF92FF92DB
:103270000F931F93CF93DF93EC017A018B01CB0166
:10328000BA0120E030E040E85FE30E949C218823FF
:103290001CF460EB74E012C0C801B70120E030E01C
:1032A00048E452E40E94EB229B01AC0160E070E62E
:1032B0008AE697E40E94A0210E94082216161706AB
:1032C00014F061E070E07D836C83CB01880F991F5F
:1032D000860F971F9F838E83DF91CF911F910F9150
:1032E000FF90EF900895FC019B011616170614F04D
:1032F00021E030E035832483C901880F991F820FB4
:10330000931F978386830895FC0182810E94A51DE7
:103310000895FC0166A977A9828120E030E040E0B1
:1033200050E00E94181E08950E948F000895CF92C9
:10333000DF92EF92FF920F931F93CF93DF938C0155
:10334000DC019E962D913C919F971C968D919C91AE
:103350001D972817390708F048C00E94F01A6B0122
:103360007C01F80182A993A9A4A9B5A9C81AD90A10
:10337000EA0AFB0AC0A9D1A9FE013796EE0FFF1F8A
:10338000E00FF11F80819181AA2797FDA095BA2FA8
:10339000C816D906EA06FB0608F451C02196D801E2
:1033A000D196DC93CE93D0972796CC0FDD1FC00F1C
:1033B000D11F88819981892B31F59E966D917C91E1
:1033C0009F976F5F7F4F9F967C936E939E971C96FF
:1033D0008D919C911D976817790748F0ED91FC91AC
:1033E0000280F381E02DC801099580E029C0C80161
:1033F00008960E943520FC01C80160810E94A8182F
:10340000F80191AB80ABF80182A993A9A4A9B5A951
:103410008C0D9D1DAE1DBF1D82AB93ABA4ABB5AB98
:1034200080A90190F081E02D80FD04C00190F08121
:10343000E02D03C00280F381E02DC801099581E0F1
:10344000DF91CF911F910F91FF90EF90DF90CF9080
:103450000895CF93DF93EC011FA61EA68C859D8552
:10346000892BD1F0CE01089660E070E00E943520F3
:10347000FC01CE0160810E94A81899AB88ABE8815D
:10348000F9810190F081E02DCE0109950E94F01A9A
:103490006AAB7BAB8CAB9DABDF91CF910895CF93A3
:1034A000DF93EC0108960E9496208C859D859FA74E
:1034B0008EA788A980FD07C0E881F9810280F38189
:1034C000E02DCE010995DF91CF910895FC01828115
:1034D00061E00E94921B0895CF92DF92EF92FF92DB
:1034E0000F931F938C0169017A0181E291E0F80149
:1034F0009183808373836283C801089665E071E0DD
:103500000E943921C801B701A6010E9436191F91F6
:103510000F91FF90EF90DF90CF900895CF92DF92C0
:10352000EF92FF920F931F937C016A01A90198010A
:103530000E946C1A89E191E0F70191838083D7AAF8
:10354000C6AA1F910F91FF90EF90DF90CF90089542
:103550001F920F920FB60F9211242F933F938F93C8
:103560009F93AF93BF938091700290917102A0914D
:103570007202B0917302309174020196A11DB11DC7
:10358000232F2D5F2D3720F02D570196A11DB11D42
:10359000209374028093700290937102A093720240
:1035A000B093730280916C0290916D02A0916E02B3
:1035B000B0916F020196A11DB11D80936C02909392
:1035C0006D02A0936E02B0936F02BF91AF919F9175
:1035D0008F913F912F910F900FBE0F901F901895D4
:1035E0008FB7F8942091700230917102409172026D
:1035F000509173028FBFB901CA0108959B01AC01BC
:103600007FB7F89480916C0290916D02A0916E0248
:10361000B0916F0266B5A89B05C06F3F19F0019687
:10362000A11DB11D7FBFBA2FA92F982F8827860F04
:10363000911DA11DB11D62E0880F991FAA1FBB1F1C
:103640006A95D1F7BC012DC0FFB7F89480916C0248
:1036500090916D02A0916E02B0916F02E6B5A89BA9
:1036600005C0EF3F19F00196A11DB11DFFBFBA2F94
:10367000A92F982F88278E0F911DA11DB11DE2E063
:10368000880F991FAA1FBB1FEA95D1F7861B970BBE
:10369000885E9340C8F2215030404040504068510D
:1036A0007C4F211531054105510571F60895789437
:1036B00084B5826084BD84B5816084BD85B5826037
:1036C00085BD85B5816085BDEEE6F0E080818160D5
:1036D0008083E1E8F0E010828081826080838081D5
:1036E00081608083E0E8F0E0808181608083E1EBAD
:1036F000F0E0808184608083E0EBF0E08081816095
:103700008083EAE7F0E0808184608083808182604A
:103710008083808181608083808180688083109233
:10372000C1000895482F50E0CA0185569F4FFC0103
:10373000249149575F4FFA0184918823C1F0E82F03
:10374000F0E0EE0FFF1FE759FF4FA591B4916623FC
:1037500041F49FB7F8948C91209582238C939FBF5E
:1037600008959FB7F8948C91822B8C939FBF0895F6
:10377000482F50E0CA0181559F4FFC012491CA0196
:1037800085569F4FFC01349149575F4FFA01949140
:10379000992309F444C0222351F1233071F02430DD
:1037A00028F42130A1F0223011F514C02630B1F0F8
:1037B0002730C1F02430D9F404C0809180008F7785
:1037C00003C0809180008F7D8093800010C084B5FD
:1037D0008F7702C084B58F7D84BD09C08091B00011
:1037E0008F7703C08091B0008F7D8093B000E92F68
:1037F000F0E0EE0FFF1FED58FF4FA591B491662347
:1038000041F49FB7F8948C91309583238C939FBF9C
:1038100008959FB7F8948C91832B8C939FBF089544
:103820001F920F920FB60F9211242F933F934F9335
:103830008F939F93EF93FF934091C600E091F50221
:10384000F091F60231969F012F7730703197809179
:10385000F7029091F8022817390739F0EB58FD4F1D
:1038600040833093F6022093F502FF91EF919F91F0
:103870008F914F913F912F910F900FBE0F901F90FE
:103880001895CF93DF93EC019A01AB01E885F98598
:10389000203081EE380780E0480780E0580709F4BF
:1038A00049C081E090E00A8802C0880F991F0A94FD
:1038B000E2F7808360E079E08DE390E00E94A3234B
:1038C0002150304040405040CA01B90122E030E070
:1038D00040E050E00E94A323EC81FD813083EE8123
:1038E000FF812083EA85FB85208141E050E0CA0109
:1038F0000E8402C0880F991F0A94E2F7282B2083B8
:10390000EA85FB852081CA010F8402C0880F991FB8
:103910000A94E2F7282B2083EA85FB8580810888BA
:1039200002C0440F551F0A94E2F7842B8083DF9175
:10393000CF910895108220E130E0CECFDC011296C5
:10394000ED91FC911397E058FF4F219131918081C7
:103950009181281B390B2F773070C9010895DC0144
:103960001296ED91FC911397EE57FF4F2081318114
:1039700092918291E058F0408217930719F42FEF4B
:103980003FEF05C0E20FF31F8081282F30E0C9010F
:103990000895DC011296ED91FC911397DF01AE576B
:1039A000BF4F2D913C911197E058FF4F808191813D
:1039B000E058F0408217930719F42FEF3FEF0BC048
:1039C000E20FF31F80812F5F3F4F2F7730702D93D1
:1039D0003C93282F30E0C9010895DC011296ED9147
:1039E000FC911397EE57FF4F8081918192938293C0
:1039F0000895FC01A085B18521898C9190E0022E6B
:103A000002C0959587950A94E2F780FFF6CF04846B
:103A1000F585E02D608308958DE491E09093FA029E
:103A20008093F90285E792E09093FC028093FB0279
:103A300085EC90E09093FE028093FD0284EC90E090
:103A4000909300038093FF0280EC90E09093020338
:103A50008093010381EC90E090930403809303032F
:103A600086EC90E0909306038093050384E08093B6
:103A7000070383E08093080387E08093090385E0D0
:103A800080930A0381E080930B0308950E94571BE3
:103A90000E942C180E94EB17FDCF0F931F93CF931A
:103AA000DF938C01EB0109C02196D801ED91FC91C7
:103AB0000190F081E02DC801099568816623A1F786
:103AC000DF91CF911F910F910895EF92FF920F9385
:103AD0001F93CF93DF938C017B01EA010CC0D701C8
:103AE0006D917D01D801ED91FC910190F081E02D67
:103AF000C80109952197209791F7DF91CF911F91E8
:103B00000F91FF90EF900895813041F0813018F0CF
:103B10008230D1F409C010926E00089580916F0038
:103B20008D7F80936F000895809170008D7F8093CA
:103B3000700081E08093B0008091B100887F846044
:103B40008093B1001092B30008951F93182F8091B5
:103B50001401811711F09FEF06C0E8E6F0E09491A0
:103B60008FEF80931401892F0E94841D812F60E0C4
:103B70000E94B81B1F9108951F920F920FB60F92CB
:103B800011242F933F934F935F936F937F938F9362
:103B90009F93AF93BF93EF93FF9380911A039091FC
:103BA0001B03A0911C03B0911D030097A105B10553
:103BB00051F1E0911E03F0911F0380819091200349
:103BC0008927808380911A0390911B03A0911C0385
:103BD000B0911D03181619061A061B06C4F480912D
:103BE0001A0390911B03A0911C03B0911D03019730
:103BF000A109B10980931A0390931B03A0931C039E
:103C0000B0931D0304C0809114010E94A51DFF9173
:103C1000EF91BF91AF919F918F917F916F915F9144
:103C20004F913F912F910F900FBE0F901F901895BD
:103C30002F923F925F926F927F928F929F92AF925C
:103C4000BF92CF92DF92EF92FF920F931F93DF9379
:103C5000CF9300D000D0CDB7DEB7A82F1B012983AA
:103C60003A834B835C83809114018A1721F4E8E640
:103C7000F0E0549082C08F3F09F0DAC1A0931401A4
:103C8000E8E6F0E054902FEF521609F4D1C181E03C
:103C9000581639F192E0591609F449C0552009F037
:103CA0006CC014BC15BC84B5826084BD85B58160D0
:103CB00085BD2A2F30E0F901E957FF4FE491F0E08C
:103CC000EE0FFF1FED58FF4F8591949190931103D4
:103CD0008093100325563F4FF9018491809312037E
:103CE0004EC0109280001092810080918100886007
:103CF00080938100809181008160809381002A2FD0
:103D000030E0F901E957FF4FE491F0E0EE0FFF1FBB
:103D1000ED58FF4F8591949190931803809317036A
:103D200025563F4FF90184918093190328C01092C2
:103D3000B0001092B1008091B00082608093B0001A
:103D40008091B10081608093B1002A2F30E0F901A9
:103D5000E957FF4FE491F0E0EE0FFF1FED58FF4FE2
:103D60008591949190931F0380931E0325563F4F96
:103D7000F90184918093200302C057FC59C18A2F16
:103D800061E00E94921B552021F0F2E05F1609F0DD
:103D9000BEC031018824992460E072E18AE790E096
:103DA000A40193010E94A32359016A0186017501B0
:103DB0000894E108F108010911092FEFE216F10456
:103DC0000105110509F008F499C060E472E48FE080
:103DD00090E0A40193010E94A32379018A01089431
:103DE000E108F1080109110982E05816C1F49FEFBA
:103DF000E916F1040105110509F008F484C060E931
:103E000070ED83E090E0A40193010E94A323790167
:103E10008A010894E108F1080109110983E0AFEF74
:103E2000EA16F1040105110509F008F468C068E418
:103E300078EE81E090E0A40193010E94A323790130
:103E40008A010894E108F10801091109552011F4CB
:103E500083E01DC0B2E05B1611F084E018C0EFEF04
:103E6000EE16F1040105110509F008F4DFC064E263
:103E700074EF80E090E0A40193010E94A3237901F4
:103E80008A010894E108F1080109110985E0FFEFB2
:103E9000EF16F1040105110591F188F162E17AE76D
:103EA00080E090E0A40193010E94A32379018A019C
:103EB0000894E108F10801091109552011F086E084
:103EC00001C084E02FEFE216F10401051105B9F0FD
:103ED000B0F0C601B50120E034E040E050E00E94BF
:103EE000A32379018A010894E108F1080109110965
:103EF000552011F087E008C085E003C081E055201F
:103F000019F485BD3AC082E08093B10036C05101FA
:103F1000CC24DD2460E072E18AE790E0A6019501FF
:103F20000E94A32379018A010894E108F10801099C
:103F3000110980E0E81680E0F80681E0080780E0DB
:103F4000180710F491E010C068E478EE81E090E08A
:103F5000A60195010E94A32379018A010894E10832
:103F6000F1080109110993E0A1E05A1631F480919A
:103F70008100887F982B9093810089819A81AB8101
:103F8000BC810097A105B10529F48FEF9FEFAFEF3A
:103F9000BFEF13C0220C331CB10180E090E02981F7
:103FA0003A814B815C810E944E2328EE33E040E051
:103FB00050E00E948123C901DA01E1E05E16A1F020
:103FC000F2E05F1619F1552099F5E7BC80930C03D8
:103FD00090930D03A0930E03B0930F0380916E0096
:103FE000826080936E0024C0F0928900E092880085
:103FF0008093130390931403A0931503B0931603B7
:1040000080916F00826080936F0012C0E092B300D5
:1040100080931A0390931B03A0931C03B0931D037A
:104020008091700082608093700002C084E06CCF49
:104030000F900F900F900F90CF91DF911F910F91E4
:10404000FF90EF90DF90CF90BF90AF909F908F90B8
:104050007F906F905F903F902F90089570E0382F81
:1040600020E0622B732BCB010895FC019B0184811E
:1040700095816817790728F4608171816115710550
:1040800029F41092210361E273E002C0620F731FF2
:10409000CB0108950F931F93CF93DF93EC018B0116
:1040A000FB01648175818C819D81680F791F7D83FF
:1040B0006C838A819B8186179707B8F46F5F7F4F67
:1040C000888199810E9491014C815D81009729F03E
:1040D000998388835B834A8308C0F8018481958132
:1040E000481B590B5D834C8307C0F80160817181C7
:1040F000888199810E946F02CE01DF91CF911F913B
:104100000F910895CF93DF93EC01CB017B836A83FA
:1041100001960E948F0099838883009721F41B8267
:104120001A821D821C82DF91CF9108950F931F93F5
:10413000CF93DF93EC018B018617970709F1FB0101
:10414000248135818C819D818217930750F4888169
:1041500099810E943901F80164817581CE010E9424
:104160008220288139812115310551F0F80184819F
:1041700095819D838C8360817181C9010E947A023F
:10418000CE01DF91CF911F910F9108951F93CF938F
:10419000DF93EC01162F81E090E09D838C83CE01AC
:1041A00061E070E00E948220E881F981309721F07F
:1041B0001083E881F9811182DF91CF911F910895D9
:1041C0000F931F93CF93DF938C01EB016C817D8163
:1041D000FC01758364830E948220F80180819181B3
:1041E000009721F0688179810E947A02DF91CF9156
:1041F0001F910F910895EF92FF920F931F93DF93FA
:10420000CF93CDB7DEB7A1970FB6F894DEBF0FBE40
:10421000CDBF8C019A0180E090E07E010894E11C02
:10422000F11CA7010E948102F70101900020E9F72B
:104230003197EE19FF09D8011596FC93EE93149768
:10424000C801BF010E948220F801808191810097FE
:1042500019F0B7010E947A02A1960FB6F894DEBF5A
:104260000FBECDBFCF91DF911F910F91FF90EF90C7
:1042700008950F931F93CF93DF938C01EB0161158A
:10428000710511F4C6E0D1E0FE0101900020E9F7CC
:104290003197EC1BFD0BD8011596FC93EE93149708
:1042A000C801BF010E948220F8018081918100979E
:1042B00019F0BE010E947A02DF91CF911F910F91F8
:1042C0000895AF92BF92CF92DF92EF92FF920F9339
:1042D0001F93CF93DF93B82EA92E6B01C82FD92F30
:1042E000FB0160817181CE010E943921EE24FF24FF
:1042F00010C0088119810E0D1F1DF80180819927BA
:1043000087FD90950E94C423F80180830894E11CE6
:10431000F11CF60184819581E816F90650F38B2D86
:104320009A2DDF91CF911F910F91FF90EF90DF9029
:10433000CF90BF90AF900895D9D008F481E0089550
:104340000CD00FC107D140F0FED030F021F45F3F18
:1043500019F0F0C0511139C1F3C014D198F3992369
:10436000C9F35523B1F3951B550BBB27AA27621739
:104370007307840738F09F5F5F4F220F331F441F7E
:10438000AA1FA9F333D00E2E3AF0E0E830D09150B6
:104390005040E695001CCAF729D0FE2F27D0660FA3
:1043A000771F881FBB1F261737074807AB07B0E8E2
:1043B00009F0BB0B802DBF01FF2793585F4F2AF0F8
:1043C0009E3F510568F0B6C000C15F3FECF3983ED8
:1043D000DCF3869577956795B795F7959F5FC9F755
:1043E000880F911D9695879597F90895E1E0660FDE
:1043F000771F881FBB1F621773078407BA0720F057
:10440000621B730B840BBA0BEE1F88F7E0950895BF
:1044100004D06894B111D9C00895BCD088F09F57DA
:1044200090F0B92F9927B751A0F0D1F0660F771F00
:10443000881F991F1AF0BA95C9F712C0B13081F0E0
:10444000C3D0B1E00895C0C0672F782F8827B85F28
:1044500039F0B93FCCF3869577956795B395D9F741
:104460003EF490958095709561957F4F8F4F9F4F4B
:104470000895E89409C097FB3EF490958095709557
:1044800061957F4F8F4F9F4F9923A9F0F92F96E9A0
:10449000BB279395F695879577956795B795F11115
:1044A000F8CFFAF4BB0F11F460FF1BC06F5F7F4FB2
:1044B0008F4F9F4F16C0882311F096E911C07723C4
:1044C00021F09EE8872F762F05C0662371F096E8CD
:1044D000862F70E060E02AF09A95660F771F881F9C
:1044E000DAF7880F9695879597F90895990F000840
:1044F000550FAA0BE0E8FEEF16161706E807F907B6
:10450000C0F012161306E407F50798F0621B730B50
:10451000840B950B39F40A2661F0232B242B252BD1
:1045200021F408950A2609F4A140A6958FEF811D74
:10453000811D089597F99F6780E870E060E0089515
:104540009FEF80EC089500240A94161617061806AB
:104550000906089500240A94121613061406050687
:104560000895092E0394000C11F4882352F0BB0F18
:1045700040F4BF2B11F460FF04C06F5F7F4F8F4F7B
:104580009F4F089557FD9058440F551F59F05F3FB6
:1045900071F04795880F97FB991F61F09F3F79F065
:1045A00087950895121613061406551FF2CF4695E7
:1045B000F1DF08C0161617061806991FF1CF869569
:1045C0007105610508940895E894BB27662777274D
:1045D000CB0197F908950BD0C4CFB5DF28F0BADF2F
:1045E00018F0952309F0A6CFABCF1124EECFCADF88
:1045F000A0F3959FD1F3950F50E0551F629FF001F6
:10460000729FBB27F00DB11D639FAA27F00DB11D4E
:10461000AA1F649F6627B00DA11D661F829F2227D7
:10462000B00DA11D621F739FB00DA11D621F839F5E
:10463000A00D611D221F749F3327A00D611D231F34
:10464000849F600D211D822F762F6A2F11249F5782
:1046500050408AF0E1F088234AF0EE0FFF1FBB1FA5
:10466000661F771F881F91505040A9F79E3F510544
:1046700070F060CFAACF5F3FECF3983EDCF38695F5
:1046800077956795B795F795E7959F5FC1F7FE2BEF
:10469000880F911D9695879597F90895629FD0018F
:1046A000739FF001829FE00DF11D649FE00DF11DED
:1046B000929FF00D839FF00D749FF00D659FF00D9C
:1046C0009927729FB00DE11DF91F639FB00DE11D89
:1046D000F91FBD01CF0111240895AA1BBB1B51E195
:1046E00007C0AA1FBB1FA617B70710F0A61BB70B62
:1046F000881F991F5A95A9F780959095BC01CD0107
:104700000895A1E21A2EAA1BBB1BFD010DC0AA1F12
:10471000BB1FEE1FFF1FA217B307E407F50720F02A
:10472000A21BB30BE40BF50B661F771F881F991FA5
:104730001A9469F760957095809590959B01AC01EE
:10474000BD01CF01089597FB092E05260ED057FD18
:1047500004D0D7DF0AD0001C38F45095409530952E
:1047600021953F4F4F4F5F4F0895F6F790958095F5
:10477000709561957F4F8F4F9F4F0895EE0FFF1FEC
:104780000590F491E02D09949111089581548A5176
:1047900008F4805E855A08952F923F924F925F925F
:1047A0006F927F928F929F92AF92BF92CF92DF9241
:1047B000EF92FF920F931F93CF93DF93CDB7DEB7A6
:1047C000CA1BDB0B0FB6F894DEBF0FBECDBF09943A
:1047D0002A88398848885F846E847D848C849B8491
:1047E000AA84B984C884DF80EE80FD800C811B819F
:1047F000AA81B981CE0FD11D0FB6F894DEBF0FBECE
:10480000CDBFED01089510E0C8ECD0E004C0FE017A
:104810000E94C0232296CA3CD107C9F7F894FFCF63
:1048200000680020000000200026030000140A0990
:1048300009FFB80BFF00000000891984190000006F
:10484000003419351905181A0C02120E1004170D30
:104850001407060F161D0A080309110B191B1C2E3D
:10486000553F4C53454B36000100000000F91C4DEC
:0C4870001D651D9E1CC91CAF1CED1C002A
:00000001FF
